:02000000C12815
:10000800A000030EA10083012D08820758291E2A8B
:10001800210E8300A00E200E090082073F3406340B
:100028005B344F3466346D347D3407347F34673441
:100038008207013402340434083482070334033459
:10004800033403349434A534C634D734E834F9344B
:100058008207013401348434843484349534A634DA
:10006800B734C834D9348207AA3437341134053444
:100078002908A90A820764340534A83402344A34AA
:100088000134A03400342908A90A82077334503493
:100098005C347C3473343E3438346D343E345C34F0
:1000A800383478345E3404345C345E34713450341B
:1000B80079346F3400343934543478340034393472
:1000C8007734733439345C340434383400346D3460
:1000D80006343D34543478346D34393400346D3456
:1000E80079345034153404345E34043421345234B1
:1000F8005834003439340F340034003473345034F5
:1001080054340034043450344F347F3473342A3434
:10011800153400340034003400346D3400340034B5
:100128006D343F3400346D343F343F340034003490
:10013800ED343F3406345B343F343F345B3466344B
:100148003F343F3466347F343F343F3467347D3442
:100158003F343F34360882071F2B632A6F2B6C2BE2
:10016800D12B9B2BC42AF62A952A572C7A2DB22DEF
:10017800DC292C2ABD299929652983163F30850059
:1001880000308600B0308700883081008312043048
:100198009200D0015014CC011D214721E830B30052
:1001A8000330B4003030B5000F218B1336083A21E4
:1001B800E9240A304624071AEF28871EDC28E92498
:1001C8000A304624071AFC28871AE328B603103099
:1001D800B61BB600D928E9240A304624871AFC2819
:1001E800071AEF28B60A3608113A0319B601D928B2
:1001F8000F21FF20AE288316051485140516051552
:10020800871707178515851606309F008312080083
:10021800231D08002311BB01BC0136086425BC0A54
:100228003A086425BC0A39086425BC0A38086425DC
:100238000800BB01BC015625B6003608EF3E03187E
:10024800B601BC0A5625BA003A08FC3E0318BA01A2
:10025800BC0A5625B900F13E0318B901BC0A562557
:10026800B8003808FC3E0318B8010800A9000310BC
:10027800A90DA90D4720C8004720C9004720CA007A
:100288004720CB000800243065230030C8005121E6
:10029800512136083A2151210800A401E9240C30E3
:1002A8004624A40B522908000B11231E602923128F
:1002B80005102C0881000C28231605142B08810032
:1002C8000C28831605108230810083120030AD009F
:1002D8008B168B173508023E65233508003CAB00AA
:1002E8003508603C003CAC000A304624E9240A305A
:1002F8004624E924B00B78291930B000053046248B
:10030800E924071E8B29871E9129B0018229871E9F
:10031800D928B50BB503B50A6E29071ED928B50A21
:100328003508603A0319B5036E2983160510831240
:10033800AA210530A400E92409304624A40B9F29EA
:100348001A23071A9C29871A9C29D9282630A40021
:1003580005141430D100D10BAF29000000000000B3
:1003680005101430D100D10BB7290000A40BAC291B
:1003780008008316051083125530BD00D1213D18A1
:1003880005143D1C0510E9244130D100D10BCA29C0
:10039800871AC229071AC229D9283D083E07BE0074
:1003A8003F07BF000310BD0C0318BD17BD070800A9
:1003B800831605108312DC30B0000530B100300818
:1003C800C0003108C100C201C301352506253230FD
:1003D800A400E9240A304624A40BED293008BC0007
:1003E8003108BB001A231322071E082A871EFD297D
:1003F800EB29071ED9280A30B0070318B10A3108BB
:10040800093A03190A2AE329871ED928F630B007C2
:10041800031CB1033108023A0319FF29E329BB0A77
:10042800BC0A051400000000BC0B162ABB0B182AD6
:10043800051008000B113308B00734080318340FEF
:10044800B107B11F0510B11B0514B73081070C287F
:10045800831605108830810083120130AD008B1798
:100468008B163308C0003408C100C201C30135250A
:1004780006253708A400E9240A304624A40B3F2A9D
:10048800FB30B7073708FB3E03184C2A0630B70085
:10049800071E582A871E522AB7013D2A071ED92847
:1004A800B30A0319B40A352A871ED928FF30B307BF
:1004B800031CB403B41F352AB301B401352A8316CB
:1004C80006309F0083123A08113E3A213A08372035
:1004D800B000752A8316051000000514831248170A
:1004E8007C2A0514051A0510083005180130C800C3
:1004F80030083C2402303C24071A852A871A6E2AC1
:10050800D828871A752A0A3046246023E924071E4A
:10051800D828871E872ABA0A3A08033C031CBA015E
:10052800672A83168713851106309F008312871365
:100538008511C80105301120C90000301120CA00FA
:10054800CB00301F48178515B322B00A301B48135B
:100558008511B322071AA92A871AA52AD928203073
:10056800A400E9240E30BB22A40BB52A0800D10050
:1005780000000000000000000000D10BBC2A0800A9
:100588008316851183128515051023141A23C001BB
:10059800C101C201C30183160514831200000000C3
:1005A8000000000000000000000000000000000043
:1005B800000000000000000000000518EB2AC00F32
:1005C800D82AC10FD82AC20FD82AC30FD82A83160F
:1005D80005108312352550245023071AF02A871A4C
:1005E800CA2AD928831685108312851023141A2342
:1005F80050304624C001C101C201C3018514000066
:10060800051C0F2BC00AC00F032BC10F032BC20FF1
:10061800032BC30F032B8510352503300425CA1778
:100628005023071A142B871AFB2AD928071087107A
:10063800071187110800831687130713A830810054
:100648000E309F0083128717071381309F00CD015A
:10065800FF308100071A332B871A332BD9288F23B1
:100668003B08283C0318402B3B08B43C031C3E2B9A
:100678004030412B7630412B38305E230B1D4A2BFE
:100688000B11FF308100B0017330C9005223B00A4A
:10069800B0080319C9012E2BA401572BA401A417D4
:1006A800572BA4012417E92406240A304624A40B56
:1006B800572B0800C800612BC801C901CA01CB012A
:1006C8000800C000C101C201C30135250625080084
:1006D80083168713702B83168E309F00831287171B
:1006E80081309F008F230310BB0CBC0C3C08C0005A
:1006F8003B08C100C201C30135250625C917C8300A
:10070800A400E9240A304624A40B852B071A762B6B
:10071800871A762BD9281F15000000001F19922B65
:1007280083161E088312BC001E08BB00080083162F
:1007380085168713051585150514A8308100063020
:100748009F00831287178101C401C501C601C70133
:10075800C823352503300425E924BD23071EB72BFC
:10076800871EA72BAC2B871ED928C8233525073011
:10077800AF2B0108C4000B1D08000B11C50F0800A2
:10078800C60F0800C70A08004408C0004508C10091
:100798004608C2004708C300080083168516871755
:1007A800051585110514A730810006309F008312B6
:1007B8000511C001C101C201C30135250625071A6B
:1007C800E92B871ED92803300425ED231624F723A7
:1007D800E12B85128101C001C101C201C301831649
:1007E8008516831208008512831685128312010864
:1007F800C100C001C003851685120108410603190E
:10080800FE2B08004D0E0339483E8400CD1B80178F
:10081800CE0A0319CF0ACF1E142C4D1B80130800D3
:1008280000000800EE30B000A730B1000000000062
:100838002A24E92406243124B00B1A2CB10B1C2CD1
:100848000830B0003124B00B262C08001030A90065
:10085800A90B2C2C0000000008000B1D382C0B11D4
:10086800C20A0319C30A08000000000000000800BB
:10087800D200D3005308D100E924D10B402CD20B6D
:100888003E2C0800D300D200D100D10B492CD20B4A
:10089800482CD30B472C08001A2524082C20CD00FF
:1008A8000F39A4000C2D83160511851085108312AD
:1008B800851007118711BF30860084242830A400D2
:1008C8000000AB24A40B642C0F30A400B424B32480
:1008D800B324AA24AA24AA24AA24AA24AA24AA2497
:1008E800AA24AA24AA240000A40B6A2C1130A4006C
:1008F800AB240000A40B7C2CA024871A612CD928D7
:100908000630A4000511D22405152E30D924A40BD5
:10091800862C0630A40005112E30D9240515D424C0
:10092800A40B8F2C0630A4000511D22405152E30F7
:10093800D924A40B982C0800D8240511CC24D5243C
:100948000515DD245930D92400000800D8240511E4
:10095800CC24D52405155D30D92400000800D824FE
:100968000511CC24D5240515CA24CA241330A9009E
:1009780000000000000000000000000085140000D6
:100988008510A90BBC2C0530D924080000000000F4
:10099800000000000000000000000000000000004F
:1009A80000000000000000000800A900A90BDA2CD4
:1009B8000800DD0A071087105D1C07145D188714EE
:1009C80000000800F03087050800F03087054C0863
:1009D800483E840000085005FF3A86004C081C2059
:1009E80087040310D00D0318FF2C0000000000003E
:1009F8000000000008005014CC0A4C19CC01080073
:100A0800A4000C2D1A2524082120CD000F39A4009C
:100A18001525C8001525C9001525CA001525CB00C0
:100A280008002408A4032425112008000930A40084
:100A380024082425003A031D0800A40B1C2D0800D7
:100A4800A9000301A91B08000310A90C2908A90D76
:100A5800543E84000008A7002918A70E27080F395C
:100A680008002030DC00D401D501D601D701D80117
:100A7800543084000530DB00333080078019F039AA
:100A8800801B0F398002840ADB0B402DC00DC10D7D
:100A9800C20DC30DD40DD50DD60DD70DD80DDC0B59
:100AA8003C2D0800831203173C088D003B088F007B
:100AB80083168C130C1483120C080313831208007A
:100AC800831203178C003C088D003B088F008316A7
:100AD8008C130C1555308D00AA308D008C14000035
:100AE80000008C18752D831203130800E624831662
:100AF800051483123808A9000310A90D3C20AE0084
:100B08003C20AF00153038073A21E924871EA72D6D
:100B1800071A892D871ED928E6254130A8001A30E2
:100B2800A5002808ED25A80A2B303C24A50B952DF7
:100B38000D30ED2564303C240A30ED25DC303C24B2
:100B4800071E892D7A2DE62414304624071ED9283D
:100B5800871EA72DB80A381123157A2D3908013EAA
:100B680065233930C8007630C9008316051483120E
:100B7800E924871EDB2D071ABC2DE6252D30AE0093
:100B8800AF0139089038ED253C30ED252830ED25AA
:100B980014303C24071ECC2D39089038ED253C3004
:100BA800ED250030ED250C21FA303C24B22D6430BF
:100BB8003C24071ED928871EDB2D2315B90A0F30C0
:100BC800B905B22DA310051CA314831605108312B2
:100BD8000800A401A415A700FF2509262718042644
:100BE800271CFF25A70CA40BF12D0926042609268E
:100BF800092609260800A31C0510A31805140800D7
:100C0800A31C0514A318051008002F08AA002E0815
:100C1800A900AA0AA90AA90B0F2EAA0B0F2E0800D1
:02400E00323F3F
:00000001FF
